:10000000F0288030A100FE30A4200130A4207530FB
:10001000A6003030BB28A101A117AE00FE30A420FD
:100020002E08A428A401A900AA01A01124080319DC
:10003000A0151030A3000301A90DAA0D031801306B
:1000400045202308031D1B280800A401A900AA01BC
:10005000A01124080319A0150530A3002730A8001B
:1000600010303E200330A800E8303E20A801643064
:100070003E20A8010A303E2029084528A7002A086A
:10008000A6002908A500CF202508A500A303031971
:10009000A011240803194F28230203185628250805
:1000A000031DA011A0195628303EA4280800AC005A
:1000B000061186118316061186110F3086058312EC
:1000C0002C08A01881283E30A6008030BB20333099
:1000D000AB0095201330A6008830BB2095206430FB
:1000E000BA2095206430BA202230AB009520283009
:1000F00080200C30802006308020A0142C0881281D
:100100002014AB00201C8F288611033C031C94286C
:1001100094200530A600DC30BB2003140800201416
:10012000FE3C0319A2288615201C201006150F304E
:1001300086052B08F03986040611AB0E2018952889
:100140003230BA202C08EB28A11B572883178001D6
:10015000840AFF3E031DA728EB28A801A700FF3053
:10016000A707031CA807031CEB280330A600DF30F9
:10017000BB20AF28A601E83EA500A609FC30031C61
:10018000C428A5070318C128A5070000A60FC12889
:100190002518CA28A51CCE280000CE280800AA01D0
:1001A000A9011030AB00260DA90DAA0D2708A90240
:1001B0002808031C280FAA020318E5282708A90706
:1001C00028080318280FAA070310A50DA60DAB0BCE
:1001D000D3282508EB28831383120313000008009B
:1001E000A00107309F00F03083168500FF308600A5
:1001F000811320308400603083128A01A720A03050
:10020000840050308A01A7202030840050308A01B9
:10021000A6200130A800F4308A01AE208A01012016
:1002200052308A01572043308A01572035308A01E5
:10023000572020308A0157204E308A0157206130E4
:100240008A0157206D308A01572065308A01572076
:1002500073308A01572020308A01572055308A0197
:1002600057204B308A01572020308A0157205630C2
:100270008A0157202D308A01572031308A015720BA
:100280008030A100C0308A010B2077308A015720CE
:100290008A0157208A0157202E308A01572070305A
:1002A0008A01572069308A01572063308A0157201C
:1002B00062308A01572061308A01572073308A01E9
:1002C000572069308A01572063308A0157202E3029
:1002D0008A0157206E308A0157206C308A015720DE
:1002E0008A119A29051A3115051E3111B60103012B
:1002F000051A013E3119013C03190130031D0301A8
:10030000B0003230360201300318030130058A1183
:1003100003198D29B60A8A017729323036028A11EB
:10032000031D94298A15E12F0430A6004C308A0160
:10033000BB20080005110510851006183114061C95
:100340003110B6018A11051EA7298A01A2290130A0
:10035000051A0301B00034303602013003180301DE
:1003600030058A110319B729B60A8A01A729343042
:1003700036028A110318BE298A15D92F3208B30014
:100380003408B50005150130A600F4308A01BB2001
:100390008A017221030131190130013A0319321324
:1003A000031D32178A017221B114311DB1108A0167
:1003B00072213416311D34128A017221B415311D97
:1003C000B4118A0172213415311D34118A01722150
:1003D000B414311DB4108A0172213414311D34104B
:1003E0008A017221B216311DB2128A0172213216AF
:1003F000311D32128A017221B215311DB2118A01EA
:1004000072213215311D32118A017221B214311D4F
:10041000B2108A0172213214311D321034083502B3
:10042000031D0130B00032083302031D01303004D7
:10043000B000060831060139031D013030048A1569
:100440000319D42F8A0101208A15061C9F2F340816
:100450008A11031D332A54308A01572056308A01ED
:1004600057208A11852C013034028A11031D432A3A
:1004700054308A01572056308A01572032308A0181
:1004800057208A11852C023034028A11031D622AFA
:1004900054308A01572065308A0157206C308A0118
:1004A000572065308A01572074308A015720653003
:1004B0008A01572078308A01572074308A015720EA
:1004C0008A11852C033034028A11031D812A56308B
:1004D0008A01572069308A01572064308A015720E9
:1004E00065308A0157206F308A01572020308A01F9
:1004F000572056308A01572044308A0157208A11EC
:10050000852C043034028A11031DA32A56308A0137
:10051000572069308A01572064308A01572065309E
:100520008A0157206F308A01572020308A015720D6
:100530004C308A01572056308A01572031308A01C9
:1005400057208A11852C053034028A11031DB62AE2
:1005500056308A01572043308A01572052308A0191
:10056000572031308A0157208A11852C06303402F9
:100570008A11031DC92A56308A01572043308A0147
:10058000572052308A01572032308A0157208A1171
:10059000852C083034028A11031DD92A53308A0170
:1005A000572041308A01572054308A0157208A1140
:1005B000852C093034028A11031DF22A43308A0146
:1005C000572061308A0157206D308A0157206530ED
:1005D0008A01572072308A01572061308A015720E2
:1005E0008A11852C0A3034028A11031D052B5330E1
:1005F0008A01572041308A01572054308A01572000
:1006000032308A0157208A11852C0C3034028A112D
:10061000031D152B43308A01572044308A0157208F
:1006200056308A0157208A11852C0D3034028A11E8
:10063000031D372B43308A01572061308A01572030
:100640006D308A01572063308A0157206F308A014C
:10065000572072308A01572064308A015720653054
:100660008A01572072308A0157208A11852C103058
:1006700034028A11031D592B41308A0157206D30F5
:100680008A01572070308A0157206C308A01572028
:1006900069308A01572066308A01572069308A0103
:1006A000572065308A01572072308A0157208A11FD
:1006B000852C113034028A11031D6F2B54308A01AE
:1006C000572075308A0157206E308A0157206530D7
:1006D0008A01572072308A0157208A11852C1230E6
:1006E00034028A11031D822B54308A015720613055
:1006F0008A01572070308A01572065308A015720BF
:100700008A11852C133034028A11031DB02B50300E
:100710008A01572072308A01572065308A0157209C
:100720002D308A01572061308A0157206D308A01AF
:10073000572070308A0157206C308A015720693069
:100740008A01572066308A01572069308A01572074
:1007500065308A01572072308A0157208A11852C12
:10076000143034028A11031DBD2B43308A015720F7
:1007700044308A0157208A11852C153034028A11A1
:10078000031DD32B50308A01572068308A0157202F
:100790006F308A0157206E308A0157206F308A01EE
:1007A00057208A11852C173034028A11031DFE2B25
:1007B00044308A01572069308A01572067308A0106
:1007C000572069308A01572074308A0157206130E0
:1007D0008A0157206C308A01572020308A01572027
:1007E00074308A01572061308A01572070308A01A5
:1007F000572065308A0157208A11852C1A3034021F
:100800008A11031D0E2C43308A01572044308A017F
:10081000572052308A0157208A11852C1D3034020E
:100820008A11031D2D2C4C308A01572069308A0112
:10083000572067308A01572068308A01572074306A
:100840008A01572069308A0157206E308A0157206B
:1008500067308A0157208A11852C1E3034028A1194
:10086000031D522C4C308A01572069308A015720D1
:1008700067308A01572068308A01572074308A0116
:10088000572069308A0157206E308A01572067301F
:100890008A01572020308A01572032308A015720A0
:1008A0008A11852C1F3034028A11031D742C543098
:1008B0008A01572065308A0157206C308A01572001
:1008C00065308A01572070308A01572068308A01CC
:1008D00057206F308A0157206E308A0157206530CB
:1008E0008A0157208A11852C53308A01572079308C
:1008F0008A01572073308A0157203A308A015720E5
:100900008030A10034088A012520C0308A010B20E4
:10091000A1010A3032028A110318A92C42308A013F
:10092000572075308A01572074308A0157208A0178
:1009300057206F308A0157206E308A0157202030AF
:100940008A0157208030A10032088A0125208A15AB
:100950009D2F0A3032028A11031DBB2C2D308A01D3
:1009600057202F308A0157202D308A0157208A01C5
:1009700057208A159D2F0B3032028A11031D172D27
:1009800034088A11031DCF2C43308A0157202F30A1
:100990008A01572050308A0157208A11152D0530C1
:1009A00034028A110319FD2C063034028A11031D0A
:1009B000FF2C43308A0157202F308A0157205030B6
:1009C0008A01572020308A0157202F308A01572072
:1009D00020308A01572053308A01572065308A0120
:1009E00057206C308A01572065308A0157206330C8
:1009F0008A01572074308A0157208A11152D14302E
:100A000034028A110319152D173034028A11031D7F
:100A1000152D54308A01572069308A0157206D30D6
:100A20008A01572065308A0157208A159D2F0C3086
:100A300032028A11031D362D53308A01572074303B
:100A40008A01572061308A0157206E308A01572071
:100A500064308A0157202D308A01572062308A0184
:100A6000572079308A0157208A159D2F0D30320288
:100A70008A11031D492D4D308A01572075308A0196
:100A8000572074308A01572065308A0157208A1513
:100A90009D2F0E3032028A11031D902D34088A11C9
:100AA000031D6C2D50308A01572065308A01572074
:100AB00072308A01572073308A0157206F308A01C3
:100AC00057206E308A01572061308A0157206C30E0
:100AD0008A0157208A118E2D053034028A1103199C
:100AE0008E2D063034028A11031D8E2D54308A015A
:100AF000572072308A01572061308A0157206330B5
:100B00008A0157206B308A01572069308A015720AB
:100B10006E308A01572067308A0157208A159D2F31
:100B20000F3032028A11031DA32D49308A0157204C
:100B30006E308A01572066308A0157206F308A0153
:100B400057208A159D2F103032028A11031DC22DA5
:100B500056308A0157206F308A0157206C308A0145
:100B6000572075308A0157206D308A015720653033
:100B70008A01572020308A0157202B308A015720C4
:100B80008A159D2F113032028A11031DE12D563036
:100B90008A0157206F308A0157206C308A01572014
:100BA00075308A0157206D308A01572065308A01DF
:100BB000572020308A0157202D308A0157208A156E
:100BC0009D2F123032028A11031D0B2E42308A01F2
:100BD000572072308A01572069308A0157206730C8
:100BE0008A01572068308A01572074308A015720C3
:100BF0006E308A01572065308A01572073308A0190
:100C000057208A01572020308A0157202B308A0133
:100C100057208A159D2F133032028A11031D352E5D
:100C200042308A01572072308A01572069308A0188
:100C3000572067308A01572068308A015720743066
:100C40008A0157206E308A01572065308A0157206B
:100C500073308A0157208A01572020308A0157209B
:100C60002D308A0157208A159D2F143032028A11A7
:100C7000031D512E43308A0157206F308A015720BF
:100C80006C308A0157206F308A01572072308A01F8
:100C9000572020308A0157202B308A0157208A158F
:100CA0009D2F153032028A11031D6D2E43308A01AB
:100CB00057206F308A0157206C308A0157206F30DF
:100CC0008A01572072308A01572020308A0157202C
:100CD0002D308A0157208A159D2F163032028A1135
:100CE000031D852E42308A01572061308A0157202A
:100CF00073308A0157208A01572020308A015720FB
:100D00002B308A0157208A159D2F173032028A1105
:100D1000031D9D2E42308A01572061308A015720E1
:100D200073308A0157208A01572020308A015720CA
:100D30002D308A0157208A159D2F183032028A11D2
:100D4000031DBC2E54308A01572072308A0157206F
:100D500065308A01572062308A0157206C308A0141
:100D6000572065308A01572020308A0157202B30C8
:100D70008A0157208A159D2F193032028A11031DCE
:100D8000DB2E54308A01572072308A01572065309B
:100D90008A01572062308A0157206C308A0157201F
:100DA00065308A01572020308A0157202D308A0172
:100DB00057208A159D2F1A3032028A11031DFD2EED
:100DC00042308A01572061308A0157206C308A01F5
:100DD000572061308A0157206E308A0157206330D6
:100DE0008A01572065308A01572020308A01572018
:100DF00052308A0157208A159D2F1B3032028A11EA
:100E0000031D1F2F42308A01572061308A0157206D
:100E10006C308A01572061308A0157206E308A0178
:100E2000572063308A01572065308A0157202030CF
:100E30008A0157204C308A0157208A159D2F1C307B
:100E400032028A11031D582F143034028A11031DF7
:100E50003F2F53308A01572068308A015720753060
:100E60008A01572066308A0157208A0157206C304A
:100E70008A01572065308A0157208A11562F173072
:100E800034028A11031D562F52308A0157206530D3
:100E90008A01572070308A01572065308A01572017
:100EA00061308A01572074308A0157208A159D2F9E
:100EB0001D3032028A11031D912F053034028A1130
:100EC0000319762F063034028A11031D782F54300F
:100ED0008A01572069308A0157206D308A015720D6
:100EE00065308A01572072308A0157208A118F2F6E
:100EF000143034028A11031D8F2F52308A0157207B
:100F000065308A01572070308A01572065308A0188
:100F1000572061308A01572074308A0157208A1582
:100F20009D2F1E3032028A11031DE22F053034023C
:100F30008A110319C12F063034028A11031DC32FF1
:100F400052308A01572065308A01572063308A0168
:100F500057206F308A01572072308A015720643041
:100F60008A01572020308A0157206D308A0157208E
:100F70006F308A01572064308A01572065308A011A
:100F800057208A11E02F113034028A11031DE02FFF
:100F900053308A01572065308A01572061308A0119
:100FA000572072308A01572063308A0157206830F9
:100FB0008A01572020308A0157202B308A01572080
:100FC0008A159D2F1F3032028A15031D3C280530DB
:100FD00034028A1503191B28063034028A15031DB2
:100FE0001D2846308A01572061308A01572073300E
:100FF0008A01572074308A01572020308A015720F7
:1010000072308A01572065308A01572076308A0174
:10101000572065308A01572072308A01572073307B
:101020008A01572065308A01572020308A015720D5
:1010300031308A0157208A153A28113034028A1536
:10104000031D3A2853308A01572065308A01572002
:1010500061308A01572072308A01572063308A013B
:10106000572068308A01572020308A0157202D30C0
:101070008A0157208A159D2F203032028A15031DC0
:101080005E2850308A01572072308A0157206F3015
:101090008A01572067308A01572072308A01572011
:1010A00061308A0157206D308A01572020308A0133
:1010B00057202B308A0157208A159D2F213032026C
:1010C0008A15031D802850308A01572072308A010A
:1010D00057206F308A01572067308A0157207230BD
:1010E0008A01572061308A0157206D308A015720CC
:1010F00020308A0157202D308A0157208A159D2FD4
:10110000223032028A15031DE02834088A15031D97
:10111000942850308A0157203C308A0157205030A3
:101120008A0157208A15DE28053034028A150319F2
:10113000C228063034028A15031DC42853308A01A0
:1011400057206C308A0157206F308A015720773042
:101150008A01572020308A01572072308A01572097
:1011600065308A01572076308A01572065308A0120
:10117000572072308A01572073308A01572065301A
:101180008A0157208A15DE28143034028A15031D7F
:10119000DE2849308A0157206E308A01572064309A
:1011A0008A01572065308A01572078308A015720FC
:1011B00020308A0157202B308A0157208A159D2F15
:1011C000233032028A15031D4F2934088A15031D66
:1011D000F62849308A0157202F308A01572049309C
:1011E0008A0157208A0157208A154D29053034027B
:1011F0008A1503191E29063034028A15031D202979
:1012000041308A01572075308A01572064308A01A5
:10121000572069308A0157206F308A0157202030CB
:101220008A0157206D308A0157206F308A0157207C
:1012300064308A01572065308A0157208A154D296C
:10124000103034028A15031D33294C308A0157208F
:1012500053308A0157202D308A01572041308A01AE
:1012600057208A154D29143034028A15031D4D2943
:1012700049308A0157206E308A01572064308A0134
:10128000572065308A01572078308A015720203056
:101290008A0157202D308A0157208A159D2F25302D
:1012A00032028A15031D772953308A015720743082
:1012B0008A01572065308A01572072308A015720F1
:1012C00065308A0157206F308A0157202F308A01FC
:1012D00057204D308A0157206F308A0157206E30D9
:1012E0008A0157206F308A0157208A159D2F273099
:1012F00032028A15031DA429053034028A15031908
:101300008F29063034028A15031D91294F308A0136
:10131000572054308A01572052308A0157208A15AD
:10132000A229103034028A15031DA2294C308A01EB
:10133000572053308A0157202D308A0157204230E0
:101340008A0157208A159D2F283032028A15031DE5
:10135000CF2953308A0157206C308A0157206F30D3
:101360008A01572077308A01572020308A01572080
:1013700046308A0157206F308A01572072308A0127
:10138000572077308A01572061308A015720723008
:101390008A01572064308A0157208A159D2F2930F1
:1013A00032028A15031D252A34088A15031DEE29E9
:1013B00054308A0157208A01572020308A01572053
:1013C00048308A0157206F308A0157206C308A01DB
:1013D000572064308A0157208A15232A05303402A9
:1013E0008A150319072A063034028A15031D092AB3
:1013F00050308A01572061308A01572075308A01A8
:10140000572073308A01572065308A0157208A158A
:10141000232A143034028A15031D232A50308A01EE
:10142000572072308A0157206F308A015720673069
:101430008A01572072308A01572061308A01572073
:101440006D308A0157208A159D2F2A3032028A1565
:10145000031DA22A34088A15031D442A54308A0128
:1014600057208A01572020308A01572054308A01A2
:10147000572069308A0157206D308A015720653026
:101480008A0157208A15A02A053034028A150319CB
:10149000782A063034028A15031D7A2A46308A01DA
:1014A000572061308A01572073308A0157207430E9
:1014B0008A01572020308A01572046308A01572060
:1014C0006F308A01572072308A01572077308A01A5
:1014D000572061308A01572072308A0157206430CA
:1014E0008A01572020308A01572031308A01572045
:1014F0008A15A02A173034028A15031DA02A5230FB
:101500008A01572065308A01572063308A015720AD
:101510006F308A01572072308A01572064308A0167
:10152000572020308A0157206D308A0157207530AE
:101530008A01572074308A01572065308A0157206C
:101540008A159D2F2B3032028A15031DD82A3408A4
:101550008A15031DCA2A54308A0157208A01572050
:1015600020308A01572045308A0157206E308A0189
:1015700057206C308A01572061308A015720723021
:101580008A01572067308A01572065308A01572029
:101590008A15D62A53308A01572063308A01572092
:1015A00061308A0157206E308A0157208A159D2F9D
:1015B0002C3032028A15031D3D2B34088A15031D79
:1015C000EE2A54308A0157208A01572020308A01A0
:1015D00057203F308A0157208A153B2B05303402B3
:1015E0008A150319222B063034028A15031D242B79
:1015F00046308A01572061308A01572073308A01B2
:10160000572074308A01572020308A0157207230C9
:101610008A01572065308A01572076308A01572089
:1016200065308A01572072308A01572073308A0151
:10163000572065308A01572020308A0157203230E8
:101640008A0157208A153B2B123034028A15031D5C
:101650003B2B44308A01572065308A015720633084
:101660008A0157206B308A01572020308A01572089
:1016700041308A0157208A159D2F2D3032028A155C
:10168000031D6D2B34088A15031D5C2B54308A0111
:1016900057208A01572020308A0157204D308A0177
:1016A000572075308A01572074308A0157206530E1
:1016B0008A0157208A156B2B45308A0157206A30E2
:1016C0008A01572065308A01572063308A015720EC
:1016D00074308A0157208A159D2F2E3032028A15C8
:1016E000031DD82B34088A15031D892B54308A0119
:1016F00057208A01572020308A0157204D308A0117
:10170000572069308A01572078308A0157208A157E
:10171000D62B053034028A150319BD2B063034024E
:101720008A15031DBF2B46308A01572061308A017C
:10173000572073308A01572074308A015720203097
:101740008A01572046308A0157206F308A0157207E
:1017500072308A01572077308A01572061308A0120
:10176000572072308A01572064308A015720203078
:101770008A01572032308A0157208A15D62B123021
:1017800034028A15031DD62B44308A015720653058
:101790008A01572063308A0157206B308A01572015
:1017A00020308A01572042308A0157208A159D2F08
:1017B0002F3032028A15031D072C143034028A158B
:1017C000031DF02B46308A01572061308A015720D3
:1017D00073308A01572074308A0157208A15052CEE
:1017E00052308A01572065308A01572076308A01AD
:1017F000572065308A01572072308A015720733094
:101800008A01572065308A0157208A159D2F303074
:1018100032028A15031D1D2C50308A015720613079
:101820008A01572075308A01572073308A0157206A
:1018300065308A0157208A159D2F313032028A1572
:10184000031D332C52308A01572065308A015720FE
:1018500073308A01572065308A01572074308A011D
:1018600057208A159D2F323032028A15031D4C2CC9
:1018700052308A01572065308A01572077308A011B
:10188000572069308A0157206E308A015720643012
:101890008A0157208A159D2F333032028A15031D85
:1018A0005F2C47308A0157206F308A01572054300F
:1018B0008A0157206F308A0157208A159D2F3430B6
:1018C00032028A15031D722C57308A015720693065
:1018D0008A0157206E308A01572064308A015720D0
:1018E0008A159D2F353032028A15031D852C503004
:1018F0008A0157206C308A01572061308A015720B5
:1019000079308A0157208A159D2F363032028A1588
:10191000031D982C53308A01572074308A015720B8
:101920006F308A01572070308A0157208A159D2F09
:10193000373032028A15031DB12C52308A015720EC
:1019400065308A01572063308A0157206F308A0141
:10195000572072308A01572064308A0157208A1537
:101960009D2F383032028A15031DCA2C45308A015A
:10197000572078308A01572074308A01572065300B
:101980008A01572072308A0157206E308A01572011
:101990008A159D2F3A3032028A15031DE02C5330F0
:1019A0008A01572050308A0157202F308A01572052
:1019B0004C308A01572050308A0157208A159D2FBC
:1019C0003C3032028A15031DFF2C54308A01572007
:1019D00065308A0157206C308A01572065308A01B2
:1019E000572074308A01572065308A01572078309B
:1019F0008A01572074308A0157208A159D2F3F3065
:101A000032028A15031D152D54308A015720563095
:101A10008A01572020308A0157206F308A015720D1
:101A20006E308A0157208A159D2F4F3032028A1559
:101A3000031D282D56308A01572069308A0157200E
:101A400065308A01572077308A0157208A159D2FEB
:101A5000503032028A15031D352D55308A0157202A
:101A600070308A0157208A159D2F513032028A1515
:101A7000031D482D44308A0157206F308A015720BA
:101A800077308A0157206E308A0157208A159D2FA2
:101A9000523032028A15031D5B2D4D308A015720CA
:101AA00065308A0157206E308A01572075308A01CF
:101AB00057208A159D2F553032028A15031D6E2D31
:101AC0004C308A01572065308A01572066308A01E0
:101AD000572074308A0157208A159D2F56303202C4
:101AE0008A15031D842D52308A01572069308A01DE
:101AF000572067308A01572068308A015720743098
:101B00008A0157208A159D2F573032028A15031DEE
:101B1000912D4F308A0157204B308A0157208A156A
:101B20009D2F5D3032028A15031DA92D46308A0192
:101B3000572072308A01572065308A0157208A0168
:101B400057207A308A01572065308A0157208A153C
:101B50009D2F613032028A15031DB92D44308A0150
:101B600057204E308A01572052308A0157208A155B
:101B70009D2F6B3032028A15031DC92D52308A0108
:101B8000572065308A01572064308A0157208A1512
:101B90009D2F6C3032028A15031DF22D34088A15F0
:101BA000031DE22D47308A01572072308A015720E9
:101BB00065308A0157208A0157206E308A015720EC
:101BC0008A15F02D143034028A15031DF02D46308D
:101BD0008A01572054308A01572053308A015720F8
:101BE0008A159D2F6D3032028A15031D0A2E593039
:101BF0008A01572065308A0157206C308A015720AE
:101C00008A0157206F308A01572077308A01572088
:101C10008A159D2F6E3032028A15031D1D2E42300B
:101C20008A0157206C308A01572075308A0157206D
:101C300065308A0157208A159D2F6F3032028A1530
:101C4000031D332E57308A01572068308A015720F0
:101C500069308A01572074308A01572065308A0123
:101C600057208A159D2F703032028A15031D4F2E82
:101C700049308A0157206E308A01572064308A012A
:101C8000572065308A01572078308A01572020304C
:101C90008A0157202B308A0157208A159D2F7130D9
:101CA00032028A15031D6B2E49308A0157206E308F
:101CB0008A01572064308A01572065308A015720F5
:101CC00078308A01572020308A0157202D308A0130
:101CD00057208A159D2F723032028A15031D962EC9
:101CE00053308A01572074308A01572061308A01AD
:101CF000572072308A01572074308A0157202030D3
:101D00008A0157206D308A01572061308A0157209F
:101D100072308A0157206B308A01572065308A0162
:101D2000572072308A0157208A159D2F7530320254
:101D30008A15031DD42E34088A15031DBC2E53307A
:101D40008A01572075308A01572062308A01572056
:101D500074308A01572069308A01572074308A0113
:101D6000572065308A0157206C308A015720733024
:101D70008A0157208A15D22E173034028A15031D86
:101D8000D22E41308A01572070308A0157208A01B3
:101D9000572065308A0157206E308A015720643001
:101DA0008A0157208A159D2F783032028A15031D2B
:101DB000EA2E46308A01572061308A01572064306C
:101DC0008A01572065308A01572072308A015720D6
:101DD0008A159D2F7A3032028A15031D362F053061
:101DE00034028A150319262F063034028A15031D82
:101DF000282F43308A0157206F308A0157207530D1
:101E00008A0157206E308A01572074308A0157208A
:101E100065308A01572072308A0157202F308A019D
:101E200057204D308A0157206F308A0157206E307D
:101E30008A01572069308A01572074308A0157205F
:101E40006F308A01572072308A0157208A15342F4B
:101E500054308A01572065308A01572078308A0132
:101E6000572074308A0157208A159D2F7E30320208
:101E70008A15031D8C2F34088A15031D6B2F5030D3
:101E80008A01572069308A01572063308A01572020
:101E900074308A01572075308A01572072308A01C8
:101EA000572065308A01572020308A01572066303C
:101EB0008A0157206F308A01572072308A015720DB
:101EC0006D308A01572061308A01572074308A01B1
:101ED00057208A158A2F053034028A1503198A2F54
:101EE000063034028A15031D8A2F43308A01572099
:101EF0006F308A01572075308A0157206E308A0171
:101F0000572074308A01572065308A01572072307B
:101F10008A0157208A159D2F43308A0157206F3040
:101F20008A0157206D308A0157203A308A015720A4
:101F30008030A10032088A0125208A15D42F533021
:101F40008A01572079308A01572073308A0157203F
:101F50003A308A0157208030A10034088A012520B8
:101F60008030A10088308A010B2034088A011220B9
:101F70008030A100C0308A010B2043308A015720F5
:101F80006F308A0157206D308A0157203A308A011C
:101F9000572032088A0125208030A100C8308A01EC
:101FA0000B2032088A0112208515B11C85118A0187
:101FB0009A2905140130A800F4308A01AE208A0164
:101FC0009A29051185140130A800F4308A01AE2049
:0C1FD0003308B2003508B4008A019A29D9
:02400E00303F41
:00000001FF
